:1000000034C07AC14DC04CC04BC04AC049C048C082
:1000100047C046C045C044C043C042C041C040C0C4
:100020003FC03EC03DC009021200010100A01409FA
:10003000040000000000000012011001FF00000891
:10004000C016DC050001010200010A03540065002E
:100050007300740012036F00620064006500760094
:100060002E00610074000403090411241FBECFE5B3
:10007000D4E0DEBFCDBF10E0A0E6B0E0EAE9F7E0F3
:1000800002C005900D92A236B107D9F720E0A2E692
:10009000B0E001C01D92AF3CB207E1F74DD37BC386
:1000A000AFCFCF93DF936091B400635067FD8AC0F8
:1000B0008091B100CCE0D0E0C81BD109C854DF4F1B
:1000C0008091B0008D3209F0C9C0683009F078C065
:1000D00083EC8093A4008AE5809361001092620013
:1000E0008881807671F0CE0105D38F3F09F460C01E
:1000F0009F81911163C09E81981708F05FC0892F7E
:100100005DC02A811092AD00998191110AC01092B0
:10011000AE002DEA30E082E03093B3002093B200CD
:10012000E7CF953029F42093B5002DEA30E0F4CFE5
:10013000963071F59B81913059F488E390E090936B
:10014000B3008093B20082E190E490936200D0CF3C
:10015000923019F486E290E0F2CF9330A9F72111A2
:1001600008C086E690E09093B3008093B20084E0EC
:10017000EBCF213019F484E590E0E1CF223021F774
:100180008AE490E09093B3008093B2008AE0DCCFE1
:10019000983051F0993019F42093B700C6CF81E020
:1001A0009A3019F280E0C1CF27EB30E081E0B4CF84
:1001B000988197FD8E8190E8909362008093600013
:1001C0001092B4008091610084FF3BC08091600078
:1001D0008F3FB9F1C82F893008F0C8E08C1B80939D
:1001E00060008091A40098E889278093A400CC2324
:1001F000E1F04091B2005091B3008091620086FF1F
:100200003FC0A5EAB0E0FA019C2F84918D9331960E
:100210009150D9F72FEF2C0F30E02F5F3F4F240F75
:10022000351F3093B3002093B2006C2F85EA90E025
:100230004CD0CC5FCC3019F08FEF80936000C0932E
:10024000610084E190B3957031F48150D9F7109238
:10025000B5001092AF00DF91CF91089580916200B8
:1002600087FFAECFCE0125D28F3F21F48EE1809360
:100270006100A6CF882309F4A3CF10926000A0CF1D
:10028000DA01E5EAF0E09C2F8D9181939150E1F73E
:10029000C1CF85B7826085BF8BB780648BBF08955F
:1002A000A82FB92F80E090E041E050EA609530E05F
:1002B00009C02D9182279795879510F0842795275F
:1002C000305EC8F36F5FA8F30895EADF8D939D93C6
:1002D0000895A6E088279927AA9569F00197E1F388
:1002E0008299FCCF829BFECF81E09927A0B3019633
:1002F00011F0A570D9F70895CF93CFB7CF93C395D9
:10030000829BE9F7829B1BC0829B19C0829B17C00E
:10031000829B15C0829B13C0DF93C2B7D091CE00E1
:10032000C093CE00CD1BC85CD1B7C23012F0D15003
:1003300003C0CF3F0AF4D395D1BFDF9141C1DF9312
:10034000C091B100DD27C854DF4F829B02C0DF910E
:10035000D9CF2F930F931F9320E8829921604F9359
:100360003F930F92829922601FEF3BE0022F220FF2
:1003700000C082990C602027087040B311F400007F
:1003800037C0B2C042FFC89540B3206800000227C2
:10039000829B0BC0287F11F040B387C040B31E7F03
:1003A000829B809902C00993E8C042FDC89540B382
:1003B00021604570829908C0B1F3217F40B309F0F4
:1003C00084C01D7F00C000C042FFC89540B32260BA
:1003D0000000829B08C0237E11F040B384C040B36C
:1003E0001B7F00C000C042FDC89540B32460099344
:1003F000829908C0277C11F040B384C040B3177FB6
:1004000000C000C042FFC89540B32860012F829B06
:1004100008C02F7811F040B384C040B30F7E00C0F5
:1004200000C042FDC89540B320611FEF829908C00B
:100430002F7111F040B384C040B30F7D00C000C0E5
:1004400042FFC89540B32062315038F0829B08C00B
:100450002F73223040B314F082C08BC00F7BC8953D
:1004600042FDC89540B32064000082998BCF2F775E
:10047000243040B30CF008C00F77000083CF42FD5A
:10048000C89540B320680000022782990AC0287FDF
:1004900011F040B38ECF40B31E7F829B809901C084
:1004A00082CF42FFC89540B32160217F829B08C064
:1004B00019F000C040B38DCF40B31D7FC89500C078
:1004C00042FDC89540B322600000829908C0237E97
:1004D00011F040B38CCF40B31B7F00C000C042FF7F
:1004E000C89540B324600993829B08C0277C11F013
:1004F00040B38CCF40B3177F00C000C042FDC89509
:1005000040B32860012F829908C02F7811F040B3C2
:100510008CCF40B30F7E00C000C042FFC89540B3EF
:1005200020611FEF829B08C02F7111F040B38CCF68
:1005300040B30F7D00C000C042FDC89540B32062AB
:100540003150B8F0829907C02F73223040B30CF0BD
:100550008CCF0F7BC89542FFC89540B32064829B27
:100560008ECF2F77243040B30CF011CF0F770000DF
:1005700086CF10E41ABF002717C03B503195C31B2C
:10058000D04010E41ABF0881033CF1F00B34E1F0D5
:100590002091AF001981110F1213EDCF093649F1E7
:1005A0000D3211F0013E39F70093B6000F903F91E4
:1005B0004F911F910F912F91DF91CAB7C6FD9FCE2A
:1005C000CF91CFBFCF9118952091B600222371F320
:1005D0001091B400112311F5343012F13093B400AE
:1005E0002093B0001091B1003BE0311B3093B1007B
:1005F00017C00091B40001308CF40AE5309161001D
:1006000034FD0FC000936100C4EAD0E00EC027950E
:1006100098F4415099F4220F0000F9CF3AE501C057
:1006200032ED032EC0E0D0E032E011B31560929AB3
:1006300011BB02B320E415E0012746E002BB279579
:1006400020F4415021F4220FF9CF012746E000C0E9
:100650003B5A02BBE0F2279528F4415029F4220FBF
:100660000000F9CF012746E0279502BB20F4415056
:1006700021F4220FF9CF012746E02991000033230E
:1006800002BB29F60A7F1091B500110FC250D0406D
:1006900002BB11F01093AF0010E41ABF046011B355
:1006A0001A7F402F4A7FC895C89502BB11BB42BB39
:1006B0007DCF40916300262F30E0240F311D21347F
:1006C00031053CF081E090916300903490F480E03B
:1006D0000895DC0180E0E82FE40F861303C0E09367
:1006E0006300F0CF9D91F0E0EC59FF4F90838F5F56
:1006F000F2CF0895FC019181913021F410926300B2
:100700008FEF0895923041F484E690E09093B30027
:100710008093B20080E40895933021F4828181BFF8
:1007200080E008959430E1F781E590E09093B30084
:100730008093B20081E008959EE088E10FB6F894BE
:10074000A89581BD0FBE91BD89E185BD83E083BDC4
:100750009CE097BB83BF9DDD8A9A80E0815099F42D
:100760008A987894A8959DDCF894F894F894F89475
:10077000F894F894F894F894F894F894F894F89419
:10078000F894F894EECFA895EFE7FCE03197F1F7F5
:0A07900000C00000E3CFF894FFCF93
:02079A00FF5A04
:00000001FF
